:1000000019C034C033C000C231C030C02FC02EC0B0
:100010002DC02CC02BC02AC047C228C027C026C074
:1000200025C098C25EC25DC25CC262C264C269C2BF
:1000300074C289C211241FBE20E0A89521BD20E012
:1000400025BFECE6F5E0A0E6B0E020E003C0C895EF
:1000500031960D92A036B207D1F7A0E6B0E020E0CD
:1000600001C01D92A639B207E1F769C100C0189519
:1000700087B9369A86B184FFFDCF0FB6F89484B164
:100080000FBE95B10895482F50E0E0E0F0E865E03C
:1000900070E820916E0030916F00442314F42E27F5
:1000A0003F27440F932F822F80709078892B41F047
:1000B000220F331F262737275F5F583070F303C0A6
:1000C000220F331FF9CF30936F0020936E000895F5
:1000D000EF92FF920F931F93CF93DF9380917E0057
:1000E0009927082F192F0E5F1F4F10926F00109243
:1000F0006E00C0E0D0E0C017D1078CF43DE7E32EDE
:1001000030E0F32ED92FC82F2296FF2DEE2D8191AE
:10011000EE2EFF2EB8DF2197C1F7D12FC02F2DE78C
:1001200030E0FD2FEC2FE20FF31F80916E009091D5
:100130006F00892F99278083CE2FDF2F80916E004B
:100140008983DF91CF911F910F91FF90EF900895D8
:100150001F9381E080937D0012E080937F00809167
:10016000740080938000809173008093810080915F
:100170009100809382008091650080938300912F8D
:100180009B5F8091620080938400809168008093DF
:10019000850090937E009CDF10937B0088E28AB9F3
:1001A0008FEF8CB91F910895982F30E0F89420E0DC
:1001B00090FF1EC0A99AAB989695AB98AB98AB9858
:1001C000AB98AB983695AB9AAB9A83B380FF01C0DE
:1001D00030682F5F283060F3A99A20E083B3992715
:1001E0008095909584FD06C02F5F203418F4F6CFDB
:1001F000A998E1CF7894832F992787FD909508954A
:100200001F93CF93DF9380E0A99A8F5F8830E0F34C
:1002100080E0AA988F5F8830E0F381E0C5DF82E458
:10022000C3DF182F80E0C0DF80E0BEDFC82FC0959D
:1002300080E0BADFD82FD095133709F46DC080E87D
:100240008093730080937400809365008093910085
:10025000AA9A1092620010926800C0FF03C080E862
:1002600080936200C3FF03C088E080936800C4FFEE
:1002700005C080916200806280936200C5FF05C066
:1002800080916200806480936200C6FF05C0809107
:100290006200886080936200CC232CF4809162001D
:1002A000816080936200D0FF05C08091620082600F
:1002B00080936200D1FF05C08091680080688093C0
:1002C0006800D2FF05C08091620082608093620066
:1002D000D3FF05C080916800806880936800D4FFD8
:1002E00005C080916800806280936800D5FF05C0DA
:1002F00080916800806180936800D6FF05C080917E
:100300006800826080936800DD23ACF4809168000F
:100310008064809368000FC080E046DF80937300A4
:1003200080E042DF8093740080E03EDF80936500D0
:1003300080E03ADF8BCFDF91CF911F910895CFE519
:10034000D2E0DEBFCDBF82E083BF8FEF81BB82BB37
:100350001ABA1BBA85E886B98FEF85BB8EEE84BBCF
:100360008BE085BD80EC83BD80E809B6082A09BE14
:100370008FE289B910927B00789480E880937300B3
:1003800080937400809365008093910010926200C6
:100390001092680084E06CDE969587959695879517
:1003A00090936D0080936C00863A90F493988091BE
:1003B0007800882331F01092780022DF02C081E0BB
:1003C0000CD080917B001816D4F3882319F702C053
:1003D000939AEDCFBDDEDECFFFCF982F992349F062
:1003E00035EA21E032BF28BF88B780FFFDCF9150AA
:1003F000C9F70895CF93C82FCC2321F084E6EDDF11
:10040000C150E1F7CF9108951F920F920FB60F924E
:1004100011248F939F93809160008150809360009E
:10042000882381F180919200815080939200809185
:100430009200882301F180916A00882389F08091DD
:100440006100882351F58CE38093610080919300D3
:1004500090919400019690939400809393001DC016
:1004600084E680936A0080916100882361F3815063
:1004700080936100E4CF83E18093920081E08093D8
:100480007800D9CF8CE08093600080916A00882347
:1004900049F2815080936A00C5CF9F918F910F9050
:1004A0000FBE0F901F9018951F920F920FB60F92CC
:1004B00011242F938F939F93AF93BF93EF93FF9349
:1004C00020917B00822F992787FD9095A92FB92F26
:1004D000F92FE82FE930F10508F03CC0EF5EFF4F3F
:1004E00009948FEF8CB92F5F20937B00929832C0D4
:1004F00080EF8CB902C085E58CB92F5F20937B001B
:1005000029C01092640080917E008C5F80939000DF
:1005100080917B008F5F80937B0090916400EDE77A
:10052000F0E0E90FF11D80818CB99F5F909364002A
:1005300080919000815080939000882359F488E046
:1005400080937B0007C010927B008FEF8CB98AE00C
:1005500080B9929AFF91EF91BF91AF919F918F9146
:0C0560002F910F900FBE0F901F90189568
:00000001FF
